:100000000C9419030C9434030C9434030C943403AF
:100010000C941A150C9434030C9434030C9434038C
:100020000C94FF140C94D7150C9434030C943403E3
:100030000C9434030C9434030C9434030C94340364
:100040000C9434030C9434030C9434030C94340354
:100050000C9434031F001111110E001F1F00111901
:100060001513001F1F001F101C1F001F1F00070873
:10007000021C001F1F000E11110E001F1F00101088
:10008000101F001F1F000708021C001F00000000B7
:100090000000000043616E63656C20546F20416274
:1000A0006F727400284F4B2920546F20436F6E7479
:1000B000696E75650043686F696365203A20004981
:1000C0006E56616C69642043686F69636500204CFB
:1000D000696768742053656E736F722020200A0070
:1000E0002054696D65202D2052544320202020206B
:1000F0000A002042757A7A65722020202020202074
:1001000020200A0020436F756E74696E67204C656D
:10011000642020200A0020426C696E6B696E6720A3
:100120004C69676874730A002054656D70205365CC
:100130006E736F72202020200A0020566F6C74208E
:100140004D6574657220202020200A0020536572BE
:1001500069616C20436F6D6D202020200A002045CE
:100160004550524F4D2044617461202020200A00E8
:10017000202020202020202020202020202020207F
:100180000A002043757272656E742054696D652093
:1001900020200A00205365742054696D65202020BA
:1001A000202020200A002053657420416C61726D6C
:1001B0002020202020200A00205669657720416CED
:1001C00061726D20202020200A0020536574205485
:1001D000696D65722020202020200A002056696564
:1001E000772054696D657220202020200A0020535A
:1001F000746F7020576174636820202020200A00EB
:1002000020202020202020202020202020202020EE
:100210000A00505245535345442043414E43454CF8
:1002200020202121210A000A48656C6C6F200020E3
:1002300042757A7A6572204F4E202121210A004CA6
:100240004544202D20504F52542041202020200092
:100250004C4544202D20504F525420410A005465F3
:100260006D70657261747572650A004C69676874B7
:100270002053656E736F720A00566F6C74204D6563
:100280007465720A00556E6B6E6F772044657669EF
:100290006365002D3D2053656C656374696F6E2046
:1002A0004D656E75203D2D003020446973636F6E7F
:1002B0006E656374004D454E552053454E54204F96
:1002C0004E20434F4D0054696D654F7574202121B8
:1002D0002100212121204572726F722021212100ED
:1002E0004572726F7220447572696E672052782071
:1002F000005265636569766564203A20004C696741
:100300006874204D65746572005265636569766531
:1003100064203A2000416C61726D20536574203A6C
:100320002000416C61726D2054696D65203A200097
:100330005365742054696D657220436F756E740047
:10034000456E746572205365636F6E6473203A2046
:1003500000456E746572204D696E75746573203A40
:100360002000456E74657220486F757273203A20C4
:100370000054696D6572205365740A0042757A7A7B
:10038000657220456E61626C65640042757A7A65BB
:10039000722044697361626C656400436F756E74AA
:1003A000696E67204C454400426C696E6B696E67EC
:1003B000204C69676874730054656D707261747560
:1003C000726500566F6C74204D6574657200416CE7
:1003D000726561647920456E61626C6564003120EC
:1003E0005669657720496E666F0032205365742028
:1003F0004E616D65004669726D7761726520566564
:100400007273696F6E203A2000506F7765722055C5
:1004100070203A20004F776E6572203A2000456EBA
:10042000746572204E616D65203A20004E616D65E5
:1004300020536176656400476F6F642042796520C0
:1004400021212100476F6F642042796520212121FD
:10045000004E616D65203A20002855502956696587
:10046000772028444E295365740056657220002079
:100470004F6E20004E6577204E616D65205361768A
:10048000656400456E7465722053656300456E7443
:100490006572204D696E00456E74657220486F75F7
:1004A000720054696D6572205365740A0054696D59
:1004B0006572204E6F74205365740A00456E746532
:1004C000722053656300456E746572204D696E003D
:1004D000456E74657220486F757200456E74657262
:1004E000204461746500456E746572204D6E7468B9
:1004F00000456E7465722059656172002855502957
:1005000020546F2053746172740A0030303A3030D6
:100510003A30302E303000507265737320416E795E
:10052000204B657920546F20537461727400284405
:100530004F574E2920546F2053746F7000203A207B
:1005400000203A200054696D65722053746F7070FA
:10055000656420202000203A2000203A20002E0050
:100560005365742054696D65203234687220466F7B
:10057000726D6174005365636F6E6473203A20007E
:1005800054696D654F757420212121004D696E7588
:10059000746573203A2000486F757273203A20000A
:1005A00044617465203A20004D6F6E7468203A20D3
:1005B0000059656172203A200057726974696E674C
:1005C00020546F2052544300212121204572726F24
:1005D0007220212121004572726F72204475726968
:1005E0006E672052780054696D65722054696D659C
:1005F0004F75740A002121212054696D65722054C1
:10060000696D654F75742021212100416C61726D07
:100610002054696D656F75740A0021212120416C99
:1006200061726D2054696D65204F75742021212100
:10063000000011241FBECFE5D4E0DEBFCDBF10E027
:10064000A0E6B0E0EAE0FAE302C005900D92A63819
:10065000B107D9F710E0A6E8B0E001C01D92A63CB2
:10066000B107E1F70C94A5030C94000000C000C092
:1006700000C000C000C000C000C000C000C000C07A
:1006800000C000C000C000C000C000C0000008954D
:10069000A198A098A998A8980895A19AE7DF1DD0DD
:1006A0000895A09AE3DFA198E1DFA098DFDFA19A87
:1006B000DDDF13D00895082EA19AD8DF802D0DD04C
:1006C000882311F002D0F8CF0895A09AA19ACEDF26
:1006D000A098CCDFA198CADF08950894881F01C0B4
:1006E000880F59F0A09A18F40000A19802C0A19AAE
:1006F00000C0BCDFA098BADFF3CFA09AA198B6DF04
:10070000A098989BFECF8827999981E0AFDF992721
:100710000895882701C081E071E0A09AA198A6DF22
:10072000A098A4DF889499990894771FB0F7A09AAD
:10073000813011F0A19801C0A19A98DFA098989BF0
:10074000FECF94DF872F99270895CCE5D4E0DEBF54
:10075000CDBF84E990E09093AE008093AD0084EA31
:1007600090E09093AA008093A90085EB90E090938D
:10077000C2008093C1008FEB90E09093AC00809317
:10078000AB008EEC90E0909396008093950080EE05
:1007900090E0909398008093970082EF90E0909380
:1007A0009A008093990084E091E090939C0080935C
:1007B0009B0086E191E090939E0080939D0088E2EB
:1007C00091E09093A00080939F008AE391E0909342
:1007D000A2008093A1008CE491E09093A400809308
:1007E000A3008EE591E09093A6008093A50080E79A
:1007F00091E09093A8008093A70082E891E0909305
:10080000B0008093AF0084E991E09093B2008093B0
:10081000B10086EA91E09093B4008093B30088EB36
:1008200091E09093B6008093B5008AEC91E09093AC
:10083000B8008093B7008CED91E09093BA0080935C
:10084000B9008EEE91E09093BC008093BB0080E0F5
:1008500092E09093BE008093BD000E945A1A80914E
:100860003C009927827090700097C9F781E090E072
:100870000E946F1C898389818F5F898380913C00EE
:100880009927827090700097C9F7698181E090E0A4
:100890000E94881C809132008460809332000E9404
:1008A00061051982789460E080E00E9405188981D2
:1008B000282F3327C901820F931FFC01EB56FF4FEE
:1008C000808191810E94061A8981282F3327C901CE
:1008D000820F931FFC01E956FF4F808191810E9496
:1008E000061A60E080E00E9405188EE30E94391825
:1008F0008091350080648093350080913500806858
:100900008093350080913200846080933200809122
:100910003200886080933200809133009927807480
:100920009070009709F023C08981882301F160E06D
:1009300080E00E940518898181508983282F332700
:10094000C901820F931FFC01EB56FF4F80819181FB
:100950000E94061A8981282F3327C901820F931F0D
:10096000FC01ED56FF4F808191810E94061A000024
:100970008091330088230CF423C08981883000F5EE
:1009800060E080E00E94051889818F5F8983282FAD
:100990003327C901820F931FFC01EB56FF4F808163
:1009A00091810E94061A8981282F3327C901820F5D
:1009B000931FFC01E956FF4F808191810E94061A26
:1009C000000080913000992784709070009709F0A2
:1009D0005FC08981282F33272A833B838A819B81AB
:1009E0008430910509F442C02A813B8125303105CC
:1009F000D4F48A819B818130910571F12A813B81F8
:100A0000223031052CF48A819B81009709F1D9CFDE
:100A10002A813B812230310511F18A819B8183300B
:100A2000910501F1CECF2A813B812630310531F18C
:100A30008A819B8186309105ECF02A813B812730A9
:100A4000310501F18A819B8188309105F1F0B9CFA0
:100A500081E00E94A506B5CF0E94ED0DB2CF0E94A5
:100A6000D605AFCF81E00E941E06ABCF80E00E948A
:100A70001E06A7CF80E00E94A506A3CF82E00E94B9
:100A8000A5069FCF0E9444089CCF0E94720C99CF6C
:100A9000000080913000992788709070009709F0CD
:100AA0000DC060E080E00E94051882E192E00E94A3
:100AB000061A80E690E00E94E119EBCF0E949F1693
:100AC000F2CECF93DF93CDB7DEB724970FB6F8946D
:100AD000DEBF0FBECDBF60E484E590E00E943A190E
:100AE00060E080E00E94051881E00E94DC178091A0
:100AF0003000992784709070009709F43DC01982E6
:100B00008981803108F023C0FE0132968081982FC0
:100B10008F5F8083892F0E9439188A81883008F07E
:100B20001A821B828B818F3F09F40DC01C828C813D
:100B30008E3108F004C08C818F5F8C83F8CF8B815D
:100B40008F5F8B83EFCF89818F5F8983D9CF87E2D6
:100B500092E00E94061A82E090E00E94301A60E063
:100B600080E00E9405188A818F5F8A838A8188309D
:100B700008F4BDCF1A82BBCF19828981883008F072
:100B80000AC080915B00992769810E943A19898186
:100B90008F5F8983F2CF0E949F1624960FB6F89438
:100BA000DEBF0FBECDBFDF91CF910895CF93DF930E
:100BB000CDB7DEB721970FB6F894DEBF0FBECDBF1D
:100BC00081E00E94DC1760E080E00E94051880EF61
:100BD000809331008FE292E00E94061A8091AD006E
:100BE0009091AE000E94061A80913000992788707B
:100BF0009070009709F419C0809132008F7E809325
:100C000032000E949F1680913200806180933200F2
:100C10000E949F1680918700882331F380912B00DA
:100C2000882314F780912C00898321960FB6F894BD
:100C3000DEBF0FBECDBFDF91CF910895CF93DF937D
:100C4000CDB7DEB722970FB6F894DEBF0FBECDBF8B
:100C5000898381E00E94DC1760E080E00E94051833
:100C600080913B008A8380EF80933A0080EA8093F2
:100C70003B008981882369F580919D0090919E00B9
:100C80000E94061A8FE392E00E94061A0E949F16A5
:100C90000E949F1690913B0080EF892780933B0034
:100CA00080913000992788709070009709F005C0F6
:100CB0008A818F7080933B003FC08091870088239A
:100CC000C1F280912B008823A4F680912C008983A7
:100CD00033C080919B0090919C000E94061A80E591
:100CE00092E00E94061A8A818F7080933B00809167
:100CF0003B008F3F09F4BDCF8A8180933B008A81FE
:100D0000805F8A830E949F168091300099278870A7
:100D10009070009709F005C08A818F7080933B0026
:100D20000BC080918700882311F380912B008823CA
:100D3000F4F680912C00898322960FB6F894DEBFDA
:100D40000FBECDBFDF91CF910895CF93DF93CDB785
:100D5000DEB725970FB6F894DEBF0FBECDBF8983EF
:100D60001C8281E00E94DC178981805C80932700CF
:100D700080EC8093260080912600992780719070E6
:100D80000097C9F3809124008A83809125008B838A
:100D90008981882321F08981823009F00EC08A81FF
:100DA0009B8120E330E0829FA001839F500D929FA2
:100DB000500D1124CA018A839B8380918700813062
:100DC00011F40E94A90760E080E00E940518898163
:100DD000882341F58EE592E00E94061A45E062E024
:100DE0008A819B810E946D1880918700882381F001
:100DF00061E083E190E00E94400C44E062E08A817F
:100E00009B810E94C50762E081E790E00E94400C50
:100E100080E20E9439188FED0E94391883E40E9405
:100E2000391878C08981813009F04BC08BE692E097
:100E30000E94061A44E060E08A819B810E946D183E
:100E400080918700882359F061E083E190E00E945F
:100E5000400C44E060E08A819B810E94C50780E0ED
:100E600094E02A813B81821B930B8A839B8380E2DF
:100E70000E9439181C828A819B818736910508F46B
:100E80000AC08C818F5F8C838A819B8186569040BB
:100E90008A839B83F0CF1D828D818A3008F03AC00F
:100EA0008C81882339F08FEF0E9439188C81815012
:100EB0008C8303C080E20E9439188D818F5F8D83FF
:100EC000EBCF8981823011F589E792E00E94061A02
:100ED00045E064E08A819B810E946D1880918700C3
:100EE000882381F061E083E190E00E94400C44E0BF
:100EF00060E08A819B810E94C50762E084E790E000
:100F00000E94400C86E50E94391804C085E892E0F2
:100F10000E94061A80918700882341F080912B005F
:100F2000882324F480912C008A830AC00E949F1693
:100F300080913000992788709070009709F018CF41
:100F400025960FB6F894DEBF0FBECDBFDF91CF91CF
:100F50000895CF93DF93CDB7DEB7000080912B00CB
:100F60009927807290700097C9F38AE080932C00D3
:100F700080912B009927807290700097C9F38DE0C3
:100F800080932C00DF91CF910895CF93DF93CDB75D
:100F9000DEB727970FB6F894DEBF0FBECDBF8983AB
:100FA0009A836B834C834AE050E06D817E81898116
:100FB0009A810E94A81C1F829F818C81981708F03B
:100FC00029C080912B009927807290700097C9F3F7
:100FD0008F81282F33278D819E81F901E80FF91F1A
:100FE000808180932C008B81882381F08B818150BC
:100FF0008B838B81882351F480912B0099278072F9
:1010000090700097C9F38EE280932C008F818F5FE0
:101010008F83D2CF27960FB6F894DEBF0FBECDBF19
:10102000DF91CF910895CF93DF93CDB7DEB72697A9
:101030000FB6F894DEBF0FBECDBF89839A83898136
:101040009A819C012B833C83019689839A83EB814F
:10105000FC8184918D838D818E83882309F40BC05C
:1010600080912B009927807290700097C9F38E8130
:1010700080932C00E4CF26960FB6F894DEBF0FBE07
:10108000CDBFDF91CF910895CF93DF93CDB7DEB77A
:101090002D970FB6F894DEBF0FBECDBF1092400063
:1010A00083E38093290088E180932A0086E8809377
:1010B000400080913000992788709070009709F463
:1010C000CEC30E94A90783E992E00E9413080E9400
:1010D000A90719828981893008F01EC080912B00F0
:1010E0009927807290700097C9F389818F5C8093F3
:1010F0002C008981282F3327C901820F931FFC01FF
:10110000EB56FF4F808191810E9413080E94A9072E
:1011100089818F5F8983DECF88EA92E00E9413087D
:101120000E94A9078091C1009091C2000E941308FB
:1011300081E00E94DC1760E080E00E94051885EBEA
:1011400092E00E94061A1092C5000E94DC14809161
:10115000C500813009F406C080912B008823BCF7BC
:1011600010924E008091C500813059F40E94A90769
:1011700086EC92E00E94130810922A0010928700D9
:1011800076C380912C00898380912B0099278071F0
:101190009070009779F480912B0099278870907057
:1011A000009741F480912B009927847090700097EC
:1011B00009F417C00E94A90782ED92E00E9413086B
:1011C00081E00E94DC1780EE92E00E94061A1092E5
:1011D0002A00809130009927887090700097C9F795
:1011E00046C30E94A90781E08093870081EF92E0C7
:1011F0000E94130880912B009927807290700097AD
:10120000C9F389818A838A8180932C0089818F70B8
:1012100089838981282F33272C873D878C859D855D
:101220008430910509F407C22C853D8525303105B0
:10123000E4F48C859D8581309105E1F12C853D8517
:101240002230310534F48C859D85009709F4F1C274
:10125000FBC22C853D8522303105B1F18C859D8501
:101260008330910509F4D8C1EFC22C853D85273024
:10127000310509F4FEC18C859D85883091056CF49B
:101280002C853D852530310509F4DFC18C859D8590
:101290008630910509F4E3C1D7C22C853D852830FD
:1012A000310509F4F0C18C859D858930910509F4DB
:1012B000F1C1CAC20E94A9078DEF92E00E941308F3
:1012C00081E00E94A506C8C20E94A9070E94A90742
:1012D00080919700909198000E9413080E94A9079E
:1012E00019828981873008F01EC080912B009927D0
:1012F000807290700097C9F389818F5C80932C0075
:101300008981282F3327C901820F931FFC01E155E2
:10131000FF4F808191810E9413080E94A907898153
:101320008F5F8983DECF8091C1009091C2000E94BF
:10133000130880912B008823E4F780912C008A8386
:1013400089E093E00E94130880912B009927807216
:1013500090700097C9F38A8189838A8180932C00D9
:101360000E94A90789818133C1F40E94DC0D80911C
:101370002B0088230CF40DC0CE0105960E947D132E
:1013800060E080E00E940518CE0105960E940F14CF
:10139000EECF80912C008A835FC28981823331F540
:1013A0000E94DC0DCE01059661E00E94E1118823C8
:1013B00021F4CE0105960E94CD1381E00E94DC1736
:1013C00080912B0088230CF40DC0CE0105960E945D
:1013D0007D1360E080E00E940518CE0105960E9412
:1013E0000F14EECF80912C008A8336C2898183331B
:1013F00021F561E08DE890E00E94E111882309F079
:101400002BC2109286001092520081E00E94C416F6
:1014100085E0809353000E94A90785E193E00E9434
:1014200013088DE890E00E940F1480912B00882310
:10143000E4F780912C008A830FC289818433A9F458
:101440000E94A90782E293E00E9413088FEF809325
:101450008C008DE890E00E940F1480912B0088236F
:10146000E4F780912C008A83F7C18981853309F0E4
:1014700093C00E94A90780E393E00E9413080E9492
:10148000A90780E493E00E94130880912B00882331
:10149000E4F780912C008F708295880F807E809376
:1014A000C00080912B008823E4F780912C00982FB6
:1014B0009F708091C000890F8093C0000E94A9078F
:1014C00081E593E00E94130880912B008823E4F7C4
:1014D00080912C008F708295880F807E8093C3004E
:1014E00080912B008823E4F780912C00982F9F7027
:1014F0008091C300890F8093C3000E94A90782E6F0
:1015000093E00E94130880912B008823E4F78091D8
:101510002C008F708295880F807E8093BF00809111
:101520002B008823E4F780912C00982F9F708091E6
:10153000BF00890F8093BF0080915F008A8390E88D
:101540008A8189238A838A81882309F47894109276
:10155000940081E08093C4008FE48093440080E491
:101560000E94C416809159008A838A8180748A837C
:101570008A81882349F4809159008A838A81805C1A
:101580008A838A818093590087E08093450081E7B0
:1015900093E00E94130860C18981863359F58091D8
:1015A0002B0088230CF422C00E94A9078091BF0061
:1015B000992742E060E00E94C50761E087E790E07C
:1015C0000E94400C8091C300992742E060E00E9495
:1015D000C50761E087E790E00E94400C8091C00061
:1015E000992742E060E00E94C507D9CF80912C0086
:1015F0008A8332C18981873331F40E94A90781E04F
:101600000E94A61029C10E94A9078091AB00909169
:10161000AC000E94130820C10E94A9078CE793E048
:101620000E9413080E94D6050E94A9078BE893E048
:101630000E94130811C10E94A9078BE993E00E9440
:10164000130881E00E941E0607C10E94A90788EACC
:1016500093E00E94130880E00E941E06FDC00E94D5
:10166000A90788EB93E00E94130880E00E94A5067A
:10167000F3C00E94A90783EC93E00E94130882E064
:101680000E94A506E9C00E94A9078EEC93E00E9483
:101690001308E2C00E94A9078091A5009091A600BE
:1016A0000E9413080E94A9078EED93E00E94130880
:1016B0000E94A9078AEE93E00E9413080E94A907DE
:1016C0008091C1009091C2000E94130880912B006C
:1016D0008823E4F780912C00898389818F70898326
:1016E0008981813009F052C080913C009927827035
:1016F00090700097C9F780E090E00E946F1C89838A
:101700000E94A90785EF93E00E9413088981992719
:1017100042E060E00E94C50780913C0099278270FA
:1017200090700097C9F781E090E00E946F1C898358
:101730000E94A90789E094E00E94130889819927F3
:1017400043E060E00E94C5070E94A90785E194E09C
:101750000E94130880913C00992782709070009736
:10176000C9F747E050E062E070E08B819C810E9405
:10177000771C67E08B819C810E94400C80912B003C
:101780008823E4F780912C00898366C089818230A8
:1017900009F040C00E94A9078EE194E00E9413085E
:1017A00019828981873008F013C080912B0088232B
:1017B000E4F78981282F33278B819C81F901E80F79
:1017C000F91F80912C00808389818F5F8983E9CF05
:1017D0008B819C81FC013796108280913C00992777
:1017E000827090700097C9F748E050E062E070E0C6
:1017F0008B819C810E94931C0E94A9078CE294E03B
:101800000E94130880912B008823E4F780912C001C
:10181000898322C00E94A9070E94A9078091AB007A
:101820009091AC000E9413080E94A9070E94A9078A
:1018300013C00E94A9071092870087E394E00E94DA
:10184000130810922A0013C00E94A9078091AB00D0
:101850009091AC000E9413080E949F162ACC0E940F
:10186000A90784E494E00E94130810922A002D96A0
:101870000FB6F894DEBF0FBECDBFDF91CF910895B4
:10188000CF93DF93CDB7DEB724970FB6F894DEBFC2
:101890000FBECDBF89839A836B831C829C818B8111
:1018A000981708F016C080912B00992780729070CD
:1018B0000097C9F38C81282F332789819A81F901F8
:1018C000E80FF91F808180932C008C818F5F8C83BF
:1018D000E5CF24960FB6F894DEBF0FBECDBFDF91E3
:1018E000CF910895CF93DF93CDB7DEB72C970FB686
:1018F000F894DEBF0FBECDBF81E594E08B879C8757
:1019000081E00E94DC1760E080E00E940518809171
:10191000A5009091A6000E94061A89E594E00E9415
:10192000061A80913000992788709070009709F40A
:101930003AC180913300992780749070009709F024
:1019400056C081E00E94DC17809130009927887092
:101950009070009709F44BC080913C0099278270E9
:1019600090700097C9F780E090E00E946F1C898317
:1019700080913C009927827090700097C9F781E0B0
:1019800090E00E946F1C8A8380913C0099278270AE
:1019900090700097C9F7CE01039648E050E062E0EE
:1019A00070E00E94771C60E080E00E9405188B8543
:1019B0009C850E94061ACE0103960E94E1198AE0D6
:1019C0000E9439188AE694E00E94061A89819927B4
:1019D00042E060E00E946D188FE694E00E94061AD3
:1019E0008A81992743E060E00E946D18ADCF809115
:1019F000330088230CF495CF81E00E94DC1780919E
:101A00003C009927827090700097C9F7CE01039629
:101A100048E050E062E070E00E94771C60E081E006
:101A20000E9405188B859C850E94061A198289815F
:101A3000873008F08DC0698180E00E940518898197
:101A4000282F3327CE010196820F931FFC01329677
:101A500081E4808380913000992784709070009792
:101A600009F470C0809133009927807490700097BA
:101A700069F58981282F3327CE010196820F931FA4
:101A8000FC01329680818A35B0F48981282F332772
:101A9000CE010196820F931FDC0112968981282FB7
:101AA0003327CE010196820F931FFC01329680816D
:101AB0008F5F8C930BC08981282F3327CE0101962D
:101AC000820F931FFC01329681E480838091330062
:101AD00088236CF18981282F3327CE010196820F4C
:101AE000931FFC01329680818234B0F08981282FC7
:101AF0003327CE010196820F931FDC011296898154
:101B0000282F3327CE010196820F931FFC013296B6
:101B1000808181508C930BC08981282F3327CE017F
:101B20000196820F931FFC0132968AE5808360E064
:101B300080E00E940518CE0103960E94E1190E94E0
:101B40009F1688CF0E949F1689818F5F89836FCFF0
:101B50001A8660E080E00E9405188B859C850E94B3
:101B6000061ACE0103960E94E1198AE00E943918F4
:101B700080913C009927827090700097C9F7CE0140
:101B8000039648E050E062E070E00E94931C84E716
:101B900094E00E94061A8091300099278870907016
:101BA0000097C9F7BECE2C960FB6F894DEBF0FBED5
:101BB000CDBFDF91CF910895CF93DF93CDB7DEB73F
:101BC0008FEF809337008FEF809338000E9454137B
:101BD0000E94AD14DF91CF910895CF93DF93CDB7DD
:101BE000DEB72A970FB6F894DEBF0FBECDBF1982BD
:101BF00060E080E00E94051881E00E94DC170E94EE
:101C00009F1680913000992788709070009709F492
:101C1000B4C180913000992784709070009709F4C6
:101C200047C060E080E00E9405188981282F332793
:101C3000C901820F931FFC01E155FF4F8081918103
:101C40000E94061A8981282F3327C901820F931F0A
:101C5000FC01EF54FF4F808191810E94061A60E0E1
:101C600080E00E9405188EE30E94391880913300AD
:101C7000882334F08981863018F489818F5F8983C5
:101C800080913300992780749070009731F4898196
:101C9000882319F0898181508983809130009927A8
:101CA00088709070009709F468C10E949F16B1CFA8
:101CB0008981282F332729873A8789859A85833018
:101CC000910509F48FC029853A852430310584F4C3
:101CD00089859A8581309105D1F129853A8522300F
:101CE00031050CF059C089859A850097A1F042C151
:101CF00029853A852530310509F4DFC089859A8523
:101D0000853091050CF481C029853A85263031054E
:101D100009F42DC12FC10E94DC0D81E00E94DC1767
:101D200080913000992788709070009709F422C143
:101D3000CE0102960E947D1360E080E00E940518AB
:101D4000CE0102960E940F140E949F16E9CF81E0F7
:101D50000E94DC17CE0102960E94C60F81E00E940D
:101D6000DC170E94DC0DCE0102960E94CD138091FB
:101D70003000992788709070009709F4FBC0CE015D
:101D800002960E947D1360E080E00E940518CE015B
:101D900002960E940F14EBCF81E00E94DC170E9494
:101DA0009F168DE890E00E94C60F1092520081E0CD
:101DB0000E94C4161092860085E08093530081E053
:101DC0000E94DC1760E080E00E9405188DE890E03A
:101DD0000E940F14809130009927887090700097AE
:101DE000C9F7C8C081E00E94DC1760E080E00E9473
:101DF00005188DE890E00E940F148091300099271B
:101E0000887090700097C9F7B5C081E00E94DC1718
:101E10000E949F1620E043E854E060E08BE30E94BC
:101E20002D108093C0000E949F1620E04DE854E0E2
:101E300060E08BE30E942D108093C3000E949F16E8
:101E400020E047E954E060E087E10E942D10809394
:101E5000BF000E949F168091C000882349F48091A2
:101E6000C300882329F48091BF00882309F482C02D
:101E70001092940081E08093C4008FE4809344002A
:101E800080E40E94C41687E08093450081E00E94B0
:101E9000DC1782EA94E00E94061A8091A9009091D2
:101EA000AA000E94061A80913000992784709070D1
:101EB0000097C9F70E949F165DC081E00E94DC1761
:101EC0008091BF00882349F48091C300882329F4BE
:101ED0008091C000882309F431C080913000992797
:101EE00088709070009709F445C060E080E00E941F
:101EF00005188091BF00992742E060E00E946D18AC
:101F00008AE30E9439188091C300992742E060E07B
:101F10000E946D188AE30E9439188091C0009927A9
:101F200042E060E00E946D188AE00E9439188091BA
:101F3000AD009091AE000E94061ACFCF81E00E94C2
:101F4000DC1760E080E00E9405188DEA94E00E94B2
:101F5000061A8091AD009091AE000E94061A809101
:101F600030009927887090700097C9F703C080E00F
:101F70000E94A6100E949F1644CE2A960FB6F8948F
:101F8000DEBF0FBECDBFDF91CF9108950F931F939A
:101F9000CF93DF93CDB7DEB722970FB6F894DEBFAD
:101FA0000FBECDBF89839A8309811A8121E04CEB52
:101FB00054E060E08BE30E942D10F80180830E94C2
:101FC0009F1609811A8121E046EC54E060E08BE322
:101FD0000E942D10F80181830E949F1609811A81A9
:101FE00021E040ED54E060E087E10E942D10F8010F
:101FF00082830E949F1609811A8121E04BED54E0F3
:1020000061E08FE10E942D10F80184830E949F16E9
:1020100009811A8121E046EE54E061E08CE00E94E3
:102020002D10F80185830E949F1609811A8121E0F5
:1020300041EF54E060E083E60E942D10F8018683B2
:102040000E949F1622960FB6F894DEBF0FBECDBF3A
:10205000DF91CF911F910F910895CF93DF93CDB76B
:10206000DEB726970FB6F894DEBF0FBECDBF8983CB
:102070006A834B835C832D838A818E8380913000B9
:10208000992784709070009709F433C080913300D1
:10209000992780749070009751F49E8189819817D8
:1020A00020F48E818F5F8E8302C08A818E8380911F
:1020B0003300882354F09E818A81891720F48E8111
:1020C00081508E8302C089818E8360E080E00E940F
:1020D00005188E81992742E060E00E946D188AE021
:1020E0000E9439188B819C810E94061A0E949F16BB
:1020F000C5CF8D818823F9F08E818A838983898178
:102100009AE0692F0E94D21C89838A819AE0692F04
:102110000E94D21C892F8A83898199278F709070A1
:102120009C0122953295307F3227207F32278A8189
:102130008F70820F8E838E81992726960FB6F89422
:10214000DEBF0FBECDBFDF91CF910895CF93DF9358
:10215000CDB7DEB72C970FB6F894DEBF0FBECDBF5C
:1021600089831A821C821D8281E00E94DC1760E054
:1021700080E00E9405188CEF94E00E94061A8BE024
:1021800095E00E94061A8981882331F00E94A907F0
:1021900087E195E00E9413080000809133009927A1
:1021A00080749070009709F40BC080918700882399
:1021B000A1F380912B00882384F780912C008B83DE
:1021C00081E00E94DC170E94DC0DCE0106960E9481
:1021D0007D138E818B838091330088230CF07EC029
:1021E000CE0106960E947D139B818E81981711F176
:1021F0008091C400882359F4109294008FE4809356
:10220000440080E40E94C41687E0809345008E81DC
:102210008B838A818F5F8A838A818C3321F41A822F
:102220008C818F5F8C838C818C3321F41C828D8117
:102230008F5F8D8360E080E00E9405188D81992773
:1022400042E060E00E946D188AE30E9439188C8198
:10225000992742E060E00E946D188AE30E943918D5
:102260008A81992742E060E00E946D188AE00E940E
:1022700039188EE295E00E94061A8981882309F4B4
:10228000AACF9A8180918C00981709F4A4CF8A81F3
:1022900080938C008D81992742E060E00E94C50701
:1022A0008DE395E00E9413088C81992742E060E05D
:1022B0000E94C50781E495E00E9413088A8199274E
:1022C00042E060E00E94C5070E94A90780912B00B0
:1022D00088230CF080CF80912C008B8381E00E94BA
:1022E000DC1760E080E00E9405188D81992742E0AC
:1022F00060E00E946D188AE30E9439188C8199274A
:1023000042E060E00E946D188AE30E9439188A81D9
:10231000992742E060E00E946D188EE20E94391811
:1023200080919400992742E060E00E946D188AE055
:102330000E94391885E495E00E94061A8981882355
:1023400079F18D81992742E060E00E94C50786E51A
:1023500095E00E9413088C81992742E060E00E947A
:10236000C5078AE595E00E9413088A81992742E013
:1023700060E00E94C5078EE595E00E9413088091F9
:102380009400992742E060E00E94C5070E94A907D7
:1023900080912B008823E4F780912C008B8308C068
:1023A0000000809130009927887090700097C9F7DD
:1023B0002C960FB6F894DEBF0FBECDBFDF91CF9144
:1023C0000895CF93DF93CDB7DEB726970FB6F89475
:1023D000DEBF0FBECDBF89839A836B8380E695E015
:1023E0000E9413080E94A90785E795E00E94130840
:1023F0001092C5000E94DC148091C500813009F460
:1024000006C080912B008823BCF710924E0080916B
:10241000C500813059F40E94A90780E895E00E9428
:10242000130881E090E08D839E83E4C00E94051331
:102430008C83E981FA818C818F708083A981BA8134
:10244000E981FA8180818295807F8C930E940513B7
:102450008C83A981BA81E981FA818C81982F9F7040
:102460008081890F8C930E94A9078CE895E00E94D7
:1024700013080E9405138C83E981FA818C818F7087
:102480008183A981BA81E981FA8181818295807FE6
:10249000FD0181830E9405138C83A981BA81E981A2
:1024A000FA818C81982F9F708181890FFD01818332
:1024B0000E94A90787E995E00E9413080E9405136E
:1024C0008C83E981FA818C818F708283A981BA81A2
:1024D000E981FA8182818295807FFD0182830E9459
:1024E00005138C83A981BA81E981FA818C81982FA7
:1024F0009F708281890FFD0182830E94A9078B81D1
:10250000882309F475C080EA95E00E9413080E94B0
:1025100005138C83E981FA818C818F708483A98172
:10252000BA81E981FA8184818295807FFD0184836B
:102530000E9405138C83A981BA81E981FA818C817B
:10254000982F9F708481890FFD0184830E94A907C1
:1025500088EA95E00E9413080E9405138C83E981A4
:10256000FA818C818F708583A981BA81E981FA8192
:1025700085818295807FFD0185830E9405138C8370
:10258000A981BA81E981FA818C81982F9F70858118
:10259000890FFD0185830E94A90781EB95E00E94C8
:1025A00013080E9405138C83E981FA818C818F7056
:1025B0008683A981BA81E981FA8186818295807FAB
:1025C000FD0186830E9405138C83A981BA81E9816C
:1025D000FA818C81982F9F708681890FFD018683F7
:1025E0000E94A90789EB95E00E9413080E94A907A1
:1025F0001D821E828D819E8126960FB6F894DEBFC5
:102600000FBECDBFDF91CF910895CF93DF93CDB7AC
:10261000DEB723970FB6F894DEBF0FBECDBF000024
:1026200080912B008823E4F780912C00898380918E
:102630002B00992780719070009779F480912B007E
:10264000992788709070009741F480912B0099270A
:1026500084709070009709F418C00E94A90788EC54
:1026600095E00E94130860E081E00E94051886ED65
:1026700095E00E94061A809130009927887090702A
:102680000097C9F71A821B8204C0898199278A831F
:102690009B838A819B8123960FB6F894DEBF0FBE81
:1026A000CDBFDF91CF910895CF93DF93CDB7DEB744
:1026B00023970FB6F894DEBF0FBECDBF0E9448032C
:1026C00080ED0E944D0389838981882329F00E942F
:1026D00065031A821B8206C00E94650381E090E0B8
:1026E0008A839B838A819B8123960FB6F894DEBFF1
:1026F0000FBECDBFDF91CF9108950F931F93CF935E
:10270000DF93CDB7DEB722970FB6F894DEBF0FBECA
:10271000CDBF89839A8380ED0E945B0380E00E9495
:102720006D0381ED0E94510309811A810E948B0380
:10273000F801808309811A810E948B03F80181834B
:1027400009811A810E948B03F801828309811A8111
:102750000E948B03F801838309811A810E948B03F5
:10276000F801848309811A810E948B03F801858313
:1027700009811A810E948903F80186830E946503FA
:1027800081E090E022960FB6F894DEBF0FBECDBF79
:10279000DF91CF911F910F910895CF93DF93CDB724
:1027A000DEB722970FB6F894DEBF0FBECDBF898388
:1027B0009A8380ED0E945B0380E00E946D03E981B3
:1027C000FA8180810E946D03E981FA8181810E94F2
:1027D0006D03E981FA8182810E946D03E981FA81AA
:1027E00083810E946D03E981FA8184810E946D03D7
:1027F000E981FA8185810E946D03E981FA818681F0
:102800000E946D030E94650381E090E022960FB65E
:10281000F894DEBF0FBECDBFDF91CF910895CF9367
:10282000DF93CDB7DEB766970FB6F894DEBF0FBE65
:10283000CDBF89839A83E981FA81828182958F70E5
:102840008370805D8B83E981FA8182818F70805DE6
:102850008C838AE38D83E981FA81818182958F70EF
:102860008770805D8E83E981FA8181818F70805DC0
:102870008F838AE38887E981FA81808182958F70CE
:102880008770805D8987E981FA8180818F70805DA2
:102890008A8780E28B871C86E981FA818481829510
:1028A0008F708370805D8D87E981FA8184818F705C
:1028B000805D8E878FE28F87E981FA81858182959D
:1028C0008F708170805D888BE981FA8185818F703E
:1028D000805D898B8FE28A8BE981FA81868182957E
:1028E0008F708F70805D8B8BE981FA8186818F700C
:1028F000805D8C8B80E28D8B1E8ACE0103960E94B8
:10290000E1198AE00E943918CE010D960E94E11962
:10291000809187008823C1F0E981FA8190918C0031
:102920008081981789F0E981FA81808180938C00F9
:10293000CE01039669E00E94400CCE010D9668E03E
:102940000E94400C0E94A90766960FB6F894DEBF5D
:102950000FBECDBFDF91CF910895CF93DF93CDB759
:10296000DEB721970FB6F894DEBF0FBECDBF80ED66
:102970000E945B0380E00E946D0381ED0E94510381
:102980000E94890389830E94650389818F778983E7
:1029900080ED0E945B0380E00E946D0389810E94AC
:1029A0006D030E94650321960FB6F894DEBF0FBE3B
:1029B000CDBFDF91CF910895CF93DF93CDB7DEB731
:1029C00021970FB6F894DEBF0FBECDBF10924D0019
:1029D00010924C0080915900898389818C5F898392
:1029E00089818093590085E080934E0021960FB62F
:1029F000F894DEBF0FBECDBFDF91CF9108951F9237
:102A00000F920FB60F9211248F93CF93DF93CDB710
:102A1000DEB78091C500882329F410924E0081E032
:102A20008093C500DF91CF918F910F900FBE0F90D3
:102A30001F9018951F920F920FB60F9211242F938B
:102A40003F934F935F936F937F938F939F93AF9336
:102A5000BF93EF93FF93CF93DF93CDB7DEB7809112
:102A600094008F5F809394008091C400882309F4C0
:102A70008BC080919400823309F07DC01092940045
:102A80008091C000882369F48091C300882371F08D
:102A90008091C30081508093C3008BE38093C0007A
:102AA00005C08091C00081508093C0008091C30018
:102AB000882361F48091BF00882341F08091BF009A
:102AC00081508093BF008BE38093C3008091BF004F
:102AD000882309F059C08091C300882309F054C0AD
:102AE0008091C000882309F04FC081E00E94DC176C
:102AF00060E080E00E94051886EE95E00E94061ACC
:102B00008091A9009091AA000E94061A80918700E6
:102B1000882361F00E94A9070E94A90785EF95E02C
:102B20000E9413080E94A9070E94A9070000809133
:102B30003000992784709070009709F414C0809138
:102B400087008823A1F380912B00882384F780914C
:102B50002C008093C4001092C40081E00E94DC1716
:102B60001092450011C0109245001092C40081E0FF
:102B70000E94DC1709C08FE48093440080E40E9427
:102B8000C41687E080934500DF91CF91FF91EF91CC
:102B9000BF91AF919F918F917F916F915F914F9175
:102BA0003F912F910F900FBE0F901F9018951F927D
:102BB0000F920FB60F9211242F933F934F935F9371
:102BC0006F937F938F939F93AF93BF93EF93FF93F5
:102BD000CF93DF93CDB7DEB72797DEBFCDBF809110
:102BE00086008F5F80938600809186008D3308F485
:102BF00087C00E94DC0DCE0101960E947D1390914A
:102C000093008F81981709F070C0909192008E8187
:102C1000981709F06AC0909191008D81981709F07A
:102C200064C090918F008B81981709F05EC09091DD
:102C30008E008A81981709F058C081E00E94DC1745
:102C400060E080E00E9405188BE096E00E94061A82
:102C500080918700882361F00E94A9070E94A9073C
:102C60008AE196E00E9413080E94A9070E94A90722
:102C700010928D0010928E0010928F001092910091
:102C800010929200109293008091A9009091AA0056
:102C90000E94061A809132008F7E809332008091CC
:102CA0003000992784709070009709F415C08091C6
:102CB00087008823A1F380912B00882384F78091DB
:102CC0002C008093860080913200806180933200D6
:102CD00081E00E94DC171CC08091320080618093EB
:102CE000320081E00E94DC1713C01092860010921F
:102CF000520081E00E94C41685E08093530008C012
:102D00001092520081E00E94C41685E08093530027
:102D10002796F894DEBFCDBFDF91CF91FF91EF9161
:102D2000BF91AF919F918F917F916F915F914F91E3
:102D30003F912F910F900FBE0F901F901895CF933A
:102D4000DF93CDB7DEB722970FB6F894DEBF0FBE84
:102D5000CDBF198289818F3F09F40DC01A828A8103
:102D60008F3F09F404C08A818F5F8A83F8CF8981FD
:102D70008F5F8983EFCF22960FB6F894DEBF0FBE28
:102D8000CDBFDF91CF910895CF93DF93CDB7DEB75D
:102D900021970FB6F894DEBF0FBECDBF898389811E
:102DA0008093590021960FB6F894DEBF0FBECDBFB9
:102DB000DF91CF910895CF93DF93CDB7DEB72497FE
:102DC0000FB6F894DEBF0FBECDBF69837A838B83C5
:102DD0009C8389819A81AB81BC810097A105B10553
:102DE00009F40CC089819A81AB81BC810197A1094A
:102DF000B10989839A83AB83BC83EBCF24960FB64A
:102E0000F894DEBF0FBECDBFDF91CF910895CF9371
:102E1000DF93CDB7DEB722970FB6F894DEBF0FBEB3
:102E2000CDBF89836A8380918900882311F40E9431
:102E30005A1A9FE780913200892380933200809153
:102E400032008F7B80933200809132008F7D80939F
:102E5000320080913800877F80933800809138005D
:102E60008D7F809338008A81813029F480913800E9
:102E700082608093380089819927807190700097D3
:102E800029F08091320080688093320089819927EF
:102E900080729070009729F0809132008064809356
:102EA00032008981992780749070009729F0809171
:102EB0003200806280933200898188232CF48091D3
:102EC0003800886080933800809138008B7F809331
:102ED000380092E09A95F1F7000080913800846004
:102EE0008093380092E09A95F1F700009FE7809177
:102EF0003200892380933200809132008F7B80934F
:102F00003200809132008F7D8093320080913800B2
:102F1000877F809338008A81823009F43EC089819E
:102F2000992781709070009729F080913200806815
:102F3000809332008981992782709070009729F0E0
:102F40008091320080648093320089819927847057
:102F50009070009729F08091320080628093320057
:102F60008981992788709070009729F080913800A6
:102F7000886080933800809138008B7F8093380080
:102F800092E09A95F1F70000809138008460809378
:102F9000380092E09A95F1F7000062E870E080E076
:102FA00090E00E94DB1622960FB6F894DEBF0FBEAB
:102FB000CDBFDF91CF910895CF93DF93CDB7DEB72B
:102FC00021970FB6F894DEBF0FBECDBF898360E0B6
:102FD00089810E9407178981813021F0898182309F
:102FE00009F00AC060E574E180E090E00E94DB1621
:102FF00010928A0010928B0021960FB6F894DEBFD3
:103000000FBECDBFDF91CF910895CF93DF93CDB7A2
:10301000DEB722970FB6F894DEBF0FBECDBF89830F
:103020006A83109288008981803120F48A818230FD
:1030300008F404C081E08093880012C08A81992737
:10304000FC01E758FF4F90818981980F80E8890F34
:103050000E94DC17898180938A008A8180938B008B
:1030600022960FB6F894DEBF0FBECDBFDF91CF9191
:103070000895CF93DF93CDB7DEB721970FB6F894BD
:10308000DEBF0FBECDBF8983809188008823E1F425
:1030900089818A3061F480918B008823A9F4809122
:1030A0008B008F5F682F80E00E9405180DC0809113
:1030B0008A00803148F461E089810E94071780917D
:1030C0008A008F5F80938A0021960FB6F894DEBF46
:1030D0000FBECDBFDF91CF910895CF93DF93CDB7D2
:1030E000DEB765970FB6F894DEBF0FBECDBF8983FC
:1030F0009A836B834C8389E0898BDE011596AA8BBA
:10310000BB8BEDE7F0E0EC8BFD8BAA89BB89EC89EA
:10311000FD89898901900D928A95E1F71E8689E0E3
:103120008F878AE0888B89819A8199235CF48981D1
:103130009A81909581959F4F89839A838DE28D83A3
:1031400081E08E8700008B818823D9F08F85282F1E
:10315000332789E090E0821B930B9C018B81992798
:103160002817390770F08F8581508F878F85282F1A
:103170003327CE010596FC01E20FF31F8EE2808318
:103180001B828F8581508F878F85282F3327CE0113
:103190000596FC01E20FF31F8889282F33278981C8
:1031A0009A81B9010E94F21C805D80838889282F52
:1031B000332789819A81B9010E94F21CCB0189834E
:1031C0009A8389819A81009721F48B81882309F45D
:1031D00004C08B81863008F4B6CF8E85888B8F85AE
:1031E000893008F023C08889282F3327CE0105961F
:1031F000DC01A20FB31F8F85282F3327CE01059640
:10320000FC01E20FF31F80818C938F85282F3327D9
:10321000CE010596FC01E20FF31F80E280838889CE
:103220008F5F888B8F858F5F8F87D9CF8C81893017
:1032300010F48C81888B1F869F858889981708F0E9
:1032400010C08F85282F3327CE010196820F931F40
:10325000FC01349680810E9439188F858F5F8F879B
:10326000EBCF65960FB6F894DEBF0FBECDBFDF91F2
:10327000CF910895CF93DF93CDB7DEB727970FB6E1
:10328000F894DEBF0FBECDBF89839A836B838B8199
:10329000883020F58B819927880F991F880F991FF7
:1032A000880F991F805C0E94DC171F828F818830F5
:1032B00008F035C089819A819C012C833D83019659
:1032C00089839A83EC81FD8184918E838E8161E074
:1032D0000E9407179F819F5F9F83E8CF80E40E9431
:1032E000DC171F828B819F81981708F018C08F818F
:1032F000803408F014C089819A819C012C833D831D
:10330000019689839A83EC81FD8184918E838E81DD
:1033100061E00E9407179F819F5F9F83E3CF6091C9
:103320008B0080918A000E94051827960FB6F894AA
:10333000DEBF0FBECDBFDF91CF910895CF93DF9356
:10334000CDB7DEB721970FB6F894DEBF0FBECDBF65
:1033500089838981823088F4698180E00E94051820
:1033600080918A00803108F004C080E20E94391800
:10337000F7CF698180E00E94051821960FB6F89476
:10338000DEBF0FBECDBFDF91CF910895CF93DF9306
:10339000CDB7DEB722970FB6F894DEBF0FBECDBF14
:1033A00080918B008A8380918A00898389819A81A8
:1033B00022960FB6F894DEBF0FBECDBFDF91CF913E
:1033C0000895CF93DF93CDB7DEB723970FB6F89468
:1033D000DEBF0FBECDBF89839A8389819A81FC01AC
:1033E000E081EB832B81019689839A83222309F460
:1033F00004C08B810E943918F0CF23960FB6F89441
:10340000DEBF0FBECDBFDF91CF910895CF93DF9385
:10341000CDB7DEB726970FB6F894DEBF0FBECDBF8F
:1034200089839A8389819A819C012B833C830196AD
:1034300089839A83EB81FC8184918D838D818E8336
:10344000882309F404C08E810E943918EBCF269698
:103450000FB6F894DEBF0FBECDBFDF91CF910895B8
:10346000CF93DF93CDB7DEB723970FB6F894DEBFC7
:103470000FBECDBF89839A8389819A819C01019671
:1034800089839A83C9010E946F1C8B838B81882357
:1034900041F08B818F3F09F404C08B810E94391861
:1034A000EBCF23960FB6F894DEBF0FBECDBFDF91F2
:1034B000CF910895CF93DF93CDB7DEB781E08093AE
:1034C00089008091370084608093370080913800B4
:1034D0008460809338008091370082608093370049
:1034E0008091310080688093310080913100806448
:1034F000809331008091310080628093310080910F
:10350000370088608093370067E574E081E090E0E1
:103510000E94DB1662E080E30E9407176FE074E30D
:1035200080E090E00E94DB1662E080E30E940717D3
:1035300062E080E30E94071762E080E20E940717C2
:1035400088E20E94DC1788E00E94DC1781E00E947C
:10355000DC1786E00E94DC178CE00E94DC17DF910C
:10356000CF910895CF93DF93CDB7DEB726970FB6EF
:10357000F894DEBF0FBECDBF89839A836B837C83B3
:103580004D835E83E981FA818B819C818083918365
:10359000E981FA818D819E8182839383E981FA8119
:1035A00016821782E981FA811482158226960FB657
:1035B000F894DEBF0FBECDBFDF91CF9108950F937A
:1035C0001F93CF93DF93CDB7DEB723970FB6F89451
:1035D000DEBF0FBECDBF89839A831B82E981FA814A
:1035E00084819581009709F43FC0E981FA81A9811E
:1035F000BA8120813181FD0186819781F901E80F2F
:10360000F91F80818B83A981BA81E981FA81868142
:1036100097810196FD0186839783E981FA81A981CB
:10362000BA8126813781FD0182819381281739076C
:1036300088F009811A81E981FA81A981BA8186819C
:103640009781FD0122813381B9010E94DE1CF801BE
:1036500086839783A981BA81E981FA8184819581E2
:103660000197FD01848395838B81992723960FB65B
:10367000F894DEBF0FBECDBFDF91CF911F910F91A8
:1036800008950F931F93CF93DF93CDB7DEB72497A1
:103690000FB6F894DEBF0FBECDBF89839A836B83CC
:1036A0007C83E981FA812B813C8184819581281773
:1036B0003907C8F5A981BA81E981FA812681378164
:1036C0008B819C81820F931FFD0186839783E98103
:1036D000FA81A981BA8126813781FD018281938196
:1036E0002817390788F009811A81E981FA81A981AF
:1036F000BA8186819781FD0122813381B9010E94BF
:10370000DE1CF80186839783A981BA81E981FA8159
:10371000248135818B819C81281B390BC901FD01D6
:103720008483958304C0E981FA81148215822496EA
:103730000FB6F894DEBF0FBECDBFDF91CF911F91C2
:103740000F9108950F931F93CF93DF93CDB7DEB7FB
:1037500024970FB6F894DEBF0FBECDBF89839A833E
:103760006B837C8309811A81E981FA812681378103
:103770008B819C81820F931FE981FA8122813381A1
:10378000B9010E94DE1C9C01F80180819181F90140
:10379000E80FF91F8081992724960FB6F894DEBFB1
:1037A0000FBECDBFDF91CF911F910F9108950F9361
:1037B0001F93CF93DF93CDB7DEB725970FB6F8945D
:1037C000DEBF0FBECDBF89839A836B83E981FA8107
:1037D000A981BA8124813581FD01828193812817D5
:1037E000390760F509811A81E981FA81A981BA81D5
:1037F00026813781FD0184819581820F931FE981A4
:10380000FA8122813381B9010E94DE1C9C01F801FA
:1038100080819181F901E80FF91F8B818083A98153
:10382000BA81E981FA81848195810196FD018483C1
:1038300095838FEF90E08C839D8302C01C821D8254
:103840008C819D8125960FB6F894DEBF0FBECDBF4B
:10385000DF91CF911F910F910895CF93DF93CDB753
:10386000DEB724970FB6F894DEBF0FBECDBF8983B5
:103870009A831B821C82E981FA81A981BA81248101
:103880003581FD01828193812817390720F481E079
:1038900090E08B839C838B819C8124960FB6F89457
:1038A000DEBF0FBECDBFDF91CF910895CF93DF93E1
:1038B000CDB7DEB722970FB6F894DEBF0FBECDBFEF
:1038C00089839A83E981FA811482158222960FB640
:1038D000F894DEBF0FBECDBFDF91CF910895E1997F
:1038E000FECF9FBB8EBBE09A99278DB308954115FB
:1038F000510569F0DC01E199FECF7FBB6EBBE09A18
:103900006F5F7F4F0DB20D9241505040B1F7089557
:10391000E199FECF9FBB8EBB6DBB0FB6F894E29AC8
:10392000E19A0FBE08954115510589F0DC018FB76A
:10393000E199FECF7FBB6EBB0D900DBAF894E29A71
:10394000E19A8FBF6F5F7F4F4150504089F70895D4
:10395000E62FF72F2E2F3F2F42307CF045326CF4AC
:10396000642F77270E94DE1C805D8A330CF0895D0E
:103970008193862F972F009799F7932F822F10828C
:103980000C94C21CDC01FC0101900020E9F7329785
:10399000AE17BF0730F47C916081708331976D93CF
:1039A000F7CF0895991B79E004C0991F961708F086
:1039B000961B881F7A95C9F780950895AA1BBB1B93
:1039C00051E107C0AA1FBB1FA617B70710F0A61B1F
:1039D000B70B881F991F5A95A9F780959095BC0140
:1039E000CD01089597FB092E07260AD077FD04D054
:1039F000E5DF06D000201AF4709561957F4F089599
:0A3A0000F6F7909581959F4F089509
:103A0A0020202020202020202020202020202020AC
:103A1A00002043002056003A000040145420202081
:063A2A00202020202020D6
:00000001FF
